:020000040800F2
:100000000028002031100008751000087510000845
:100010007510000875100008751000080000000039
:100020000000000000000000000000007510000843
:10003000751000080000000075100008150F00087A
:10004000751000087510000875100008751000087C
:10005000751000087510000875100008751000086C
:10006000751000087510000875100008751000085C
:10007000751000087510000875100008751000084C
:10008000751000087510000875100008751000083C
:10009000751000087510000875100008751000082C
:1000A000751000087510000875100008751000081C
:1000B0007510000875100008000000007510000899
:1000C0007510000800000000000000007510000816
:1000D0000000000075100008751000080000000006
:1000E0007510000875100008751000080000000069
:1000F0000000000000000000000000000000000000
:0C01000000000000000000005FF808F1A3
:10010C0080B483B000AF03463960FB7197F90730B8
:10011C00002B0BDA0D49FB7903F00F03043B3A6813
:10012C00D2B21201D2B20B441A7609E0084997F9FF
:10013C0007303A68D2B21201D2B20B4483F80023D2
:10014C0000BF0C37BD4680BC704700BF00ED00E01F
:10015C0000E100E080B582B000AF78607B68B3F15D
:10016C00807F01D3012311E00A4A7B6823F07F438F
:10017C00013B53600F214FF0FF30FFF7C1FF054BE0
:10018C0000229A60034B07221A6000231846083796
:10019C00BD4680BD10E000E080B500AF154A154BA0
:1001AC001B6843F0010313601249124B5A68124B3F
:1001BC0013404B600F4A0F4B1B6823F0847323F4DE
:1001CC00803313600B4A0B4B1B6823F480231360A2
:1001DC00084A084B5B6823F4FE035360054B4FF44D
:1001EC001F029A6000F078F8044B4FF000629A609E
:1001FC0000BF80BD001002400000FFF800ED00E0E1
:10020C0080B485B000AF0023FB600023BB600023EB
:10021C007B602C4B5B6803F00C03FB60FB68042BCE
:10022C0007D0082B09D0002B33D1274B274A1A6053
:10023C0033E0254B254A1A602FE0224B5B6803F410
:10024C007013BB601F4B5B6803F480337B60BB682F
:10025C009B0C0233BB607B68002B06D1BB681C4A2D
:10026C0002FB03F3184A136017E0164B5B6803F4A8
:10027C000033002B06D0BB68154A02FB03F3124A6D
:10028C0013600AE0BB68114A02FB03F30E4A1360C9
:10029C0003E00D4B0D4A1A6000BF0A4B5B6803F07C
:1002AC00F0031B090B4AD35CDBB2FB60064B1A68EC
:1002BC00FB6822FA03F3044A136000BF1437BD46EF
:1002CC0080BC7047001002400000002000127A0031
:1002DC0000093D000400002080B500AF00F002F8DA
:1002EC0000BF80BD80B483B000AF00237B600023CF
:1002FC003B603A4A394B1B6843F480331360374BED
:10030C001B6803F400333B607B6801337B603B6804
:10031C00002B03D17B68B3F5A06FF0D12F4B1B687A
:10032C0003F40033002B02D001233B6001E00023D7
:10033C003B603B68012B4BD1294A294B1B6843F08E
:10034C0010031360264A264B1B6823F0030313602B
:10035C00234A234B1B6843F0020313601F4A1F4BB5
:10036C005B6853601D4A1D4B5B6853601B4A1B4BFB
:10037C005B6843F480635360184A184B5B6823F442
:10038C007C135360154A154B5B6843F4E8135360B8
:10039C00124A124B1B6843F08073136000BF0F4B63
:1003AC001B6803F00073002BF9D00C4A0B4B5B68F5
:1003BC0023F003035360094A084B5B6843F00203C4
:1003CC00536000BF054B5B6803F00C03082BF9D19D
:1003DC0000BF0C37BD4680BC704700BF0010024008
:1003EC000020024080B489B000AF786039600023EF
:1003FC00FB6100233B610023BB610023FB600023F6
:10040C007B610023BB603B68DB7803F00F03FB616F
:10041C003B68DB7803F01003002B05D03B689B781E
:10042C001A46FB691343FB613B681B88DBB2002B4C
:10043C0044D07B681B687B610023BB6138E00122E0
:10044C00BB6902FA03F3FB603B681B881A46FB6826
:10045C0013403B613A69FB689A4226D1BB699B0009
:10046C00FB600F22FB6802FA03F3BB60BB68DB4343
:10047C007A6913407B61FA69FB6802FA03F37A69C3
:10048C0013437B613B68DB78282B05D10122BB69C8
:10049C009A407B685A6108E03B68DB78482B04D1B2
:1004AC000122BB699A407B681A61BB690133BB614D
:1004BC00BB69072BC3D97B687A691A603B681B88B8
:1004CC00FF2B46D97B685B687B610023BB613AE0FC
:1004DC00BB690833012202FA03F3FB603B681B88FB
:1004EC001A46FB6813403B613A69FB689A4227D174
:1004FC00BB699B00FB600F22FB6802FA03F3BB6035
:10050C00BB68DB437A6913407B61FA69FB6802FACA
:10051C0003F37A6913437B613B68DB78282B05D1A5
:10052C00BB69083301229A407B685A613B68DB78CF
:10053C00482B05D1BB69083301229A407B681A61AC
:10054C00BB690133BB61BB69072BC1D97B687A6975
:10055C005A6000BF2437BD4680BC704780B483B05E
:10056C0000AF78600B467B807A887B681A6100BF8D
:10057C000C37BD4680BC704780B483B000AF786048
:10058C000B467B807A887B685A6100BF0C37BD466E
:10059C0080BC704780B483B000AF78600B46FB70B2
:1005AC00FB78002B06D00949084B9A697B681343EA
:1005BC008B6106E00549054B9A697B68DB43134068
:1005CC008B6100BF0C37BD4680BC704700100240E9
:1005DC0080B485B000AF78600B467B800023FB7342
:1005EC007B681B899AB27B8813409BB2002B02D08C
:1005FC000123FB7301E00023FB73FB7B18461437CC
:10060C00BD4680BC704700BF80B483B000AF78603B
:10061C000B467B807B687A889A8100BF0C37BD467D
:10062C0080BC704780B483B000AF78607B689B89D6
:10063C009BB218460C37BD4680BC704780B485B061
:10064C0000AF786039600023FB817B681B88FB81DD
:10065C00FB8903F44153FB813B681A883B685B8838
:10066C0013439AB23B689B8813439AB23B68DB886E
:10067C0013439AB23B681B8913439AB23B685B895C
:10068C0013439AB23B689B8913439AB23B68DB894C
:10069C0013439AB2FB891343FB817B68FA891A8056
:1006AC007B689B8B9BB223F400639AB27B689A8322
:1006BC003B681A8A7B681A8200BF1437BD4680BC1F
:1006CC00704700BF80B483B000AF78600B46FB70FE
:1006DC00FB78002B08D07B681B889BB243F040034F
:1006EC009AB27B681A8007E07B681B889BB223F068
:1006FC0040039AB27B681A8000BF0C37BD4680BCA1
:10070C00704700BF80B483B000AF78600B46FB70BD
:10071C00FB78002B06D07B689B6843F001027B685A
:10072C009A6005E07B689B6823F001027B689A6005
:10073C0000BF0C37BD4680BC704700BF80B483B08F
:10074C0000AF78607B689B6843F008027B689A6016
:10075C0000BF0C37BD4680BC704700BF80B485B06D
:10076C0000AF78600023FB737B689B6803F0080381
:10077C00002B02D00123FB7301E00023FB73FB7BF6
:10078C0018461437BD4680BC704700BF80B483B098
:10079C0000AF78607B689B6843F004027B689A60CA
:1007AC0000BF0C37BD4680BC704700BF80B485B01D
:1007BC0000AF78600023FB737B689B6803F0040335
:1007CC00002B02D00123FB7301E00023FB73FB7BA6
:1007DC0018461437BD4680BC704700BF80B483B048
:1007EC0000AF78600B46FB70FB78002B06D07B6863
:1007FC009B6843F4A0027B689A6005E07B689B6869
:10080C0023F4A0027B689A6000BF0C37BD4680BC05
:10081C00704700BF80B485B000AF786039600023AA
:10082C00FB600023FB727B685B68FB60FB6803F476
:10083C004153FB603B681A683B681B791B021343EE
:10084C00FA681343FB607B68FA685A607B689B68A4
:10085C00FB60FA68164B1340FB603B68DA683B6838
:10086C009B681A433B685B795B001343FA6813433C
:10087C00FB607B68FA689A607B68DB6AFB60FB68EC
:10088C0023F47003FB603B681B7C013BDAB2FB7A00
:10089C001343FB72FB7A1B05FA681343FB607B68FE
:1008AC00FA68DA6200BF1437BD4680BC704700BFDF
:1008BC00FDF7F1FF80B483B000AF78607B68DB6C30
:1008CC009BB218460C37BD4680BC704780B582B0D1
:1008DC0000AF0346FB7100BF02210E48FFF778FE04
:1008EC000346002BF8D0FB799BB219460948FFF759
:1008FC008BFE00BF01210748FFF76AFE0346002B61
:10090C00F8D00448FFF78EFE0346DBB218460837D2
:10091C00BD4680BD0038004080B586B000AF0121D7
:10092C000420FFF737FE01214FF48050FFF732FE11
:10093C004FF46043BB820323BB751823FB7507F18F
:10094C00140319461748FFF74DFD4FF48053BB8233
:10095C001023FB7507F1140319461248FFF742FDEB
:10096C0000233B804FF482737B800023BB800223E7
:10097C00FB8001233B814FF400737B810023BB81FF
:10098C000023FB8107233B823B4619460648FFF7B1
:10099C0055FE01210448FFF795FE00BF1837BD46F0
:1009AC0080BD00BF000C01400038004080B500AF96
:1009BC004FF480511948FFF7DFFD952200210020EC
:1009CC0000F02EF8012000F061F80346002B01D056
:1009DC00FF2320E04FF480511048FFF7BFFDFF20AC
:1009EC00FFF774FF4FF480510C48FFF7C5FDFF2251
:1009FC000021012000F014F8002000F047F8034615
:100A0C00002BE7D14FF480510448FFF7A7FDFF20DE
:100A1C00FFF75CFF0023184680BD00BF000C0140AF
:100A2C0080B586B000AF03463960FB711346BB71CD
:100A3C0000237B61FB7943F04003DBB23B733B68E3
:100A4C001B0EDBB27B733B681B0CDBB2BB733B68CE
:100A5C001B0ADBB2FB733B68DBB23B74BB797B7468
:100A6C0000237B610AE007F10C027B6913441B78BD
:100A7C001846FFF72BFF7B6901337B617B69052BE4
:100A8C00F1D900BF1837BD4680BD00BF80B584B01A
:100A9C0000AF0346FB7140F6FF73FB6002E0FB689E
:100AAC00013BFB6000F012F803461A46FB799342B7
:100ABC0002D0FB68002BF2D1FB68002B01D1FF2385
:100ACC0000E0002318461037BD4680BD80B582B0CB
:100ADC0000AF0023FB7100BF02210E48FFF778FD29
:100AEC000346002BF8D0FF210A48FFF78DFD00BF0D
:100AFC0001210848FFF76CFD0346002BF8D0054890
:100B0C00FFF790FD0346FB71FB7918460837BD468D
:100B1C0080BD00BF0038004080B582B000AF00231C
:100B2C007B601EE0FFF7D2FF0346FB70FB7803F0FF
:100B3C001F03FB70FB780B2B06D00D2B06D0052B5F
:100B4C0006D10523BB7006E00B2316E00D2314E041
:100B5C00FF23BB7000BFBB78052B06D07B6801332D
:100B6C007B607B68402BDDD900E000BF00BFFFF746
:100B7C00ADFF0346002BFAD0FB7818460837BD466C
:100B8C0080BD00BF80B582B000AF00237B60FFF753
:100B9C00C3FE4FF480510B48FFF7E0FC00237B6051
:100BAC0005E0FF20FFF792FE7B6801337B607B68DA
:100BBC00092BF6D9FFF7FAFE034618460837BD464F
:100BCC0080BD00BF000C014080B500AF094B1B88F5
:100BDC00002B01D100230AE0FFF7D4FF03469AB2A1
:100BEC00044B1A80034B1B88002BF5D101231846AC
:100BFC0080BD00BF1800002080B500AF00BFFFF71C
:100C0C00E3FF0346002BFAD100BF80BD80B586B050
:100C1C0000AFF860B9601346FB8000237B61FF23B3
:100C2C00FB744FF480511F48FFF7A6FCFF22B968F4
:100C3C001820FFF7F5FE0020FFF728FF0346002BD6
:100C4C0022D1FF20FFF742FEFE20FFF73FFE0023DC
:100C5C007B610AE0FB681B781846FFF737FEFB68E0
:100C6C000133FB607B6901337B61FA887B699A42B3
:100C7C00F0D8FFF72BFFFFF729FFFFF74DFF0346D7
:100C8C00052B01D10023FB744FF480510548FFF76D
:100C9C0065FCFF20FFF71AFEFB7C18461837BD4693
:100CAC0080BD00BF000C014080B584B000AF7860FF
:100CBC003C4B1A783C4B1A703A4B00221A700023AA
:100CCC00FB60FF23FB724FF480513848FFF754FC54
:100CDC00FF2279681820FFF7A3FE0020FFF7D6FE4D
:100CEC000346002B4ED1FF20FFF7F0FDFE20FFF74F
:100CFC00EDFD2D4B1B78012B1AD10023FB6014E06A
:100D0C002B4AFB6832F81330DBB21846FFF7DEFDD6
:100D1C00274AFB6832F813301B0A9BB2DBB2184629
:100D2C00FFF7D4FDFB680133FB60FB68FF2BE7D9B1
:100D3C001D4B1B78022B1AD10023FB6014E01D4ABB
:100D4C00FB6832F81330DBB21846FFF7BFFD194AC7
:100D5C00FB6832F813301B0A9BB2DBB21846FFF764
:100D6C00B5FDFB680133FB60FB68FF2BE7D9FFF790
:100D7C00ADFEFFF7ABFEFFF7CFFE0346052B01D10F
:100D8C000023FB724FF480510848FFF7E7FBFF206C
:100D9C00FFF79CFD044B00221A70FB7A18461037A3
:100DAC00BD4680BD300600201B000020000C014019
:100DBC00300200203004002080B586B000AF012145
:100DCC004FF40070FFF7E6FB01233B800023FB7020
:100DDC000223BB703B4619461A48FFF703FB00235E
:100DEC007B6001233B7201237B724FF46023FB6019
:100DFC0000233B6100233B753B1D19461248FFF74E
:100E0C0009FD01211048FFF77DFC0F48FFF796FC08
:100E1C0000BF0D48FFF7A2FC0346002BF9D10A488E
:100E2C00FFF7B4FC00BF0848FFF7C0FC0346002BDB
:100E3C00F9D101210448FFF7D1FC00BF1837BD469A
:100E4C0080BD00BF000801400024014080B500AF08
:100E5C004FF400720021094800F080F92322084960
:100E6C00064800F003F90020FFF71EFF03469AB274
:100E7C00044B1A800123184680BD00BF30020020AD
:100E8C005C1200081800002080B500AFFFF77AFE56
:100E9C0003461A46154B1A60FFF7AEFE144B0022A0
:100EAC001A80144B4FF400721A60FFF7A9F9124B19
:100EBC001B68124AA2FB03231B0B1846FFF74AF9C7
:100ECC00FFF77AFF0E4B1B78002BFBD00D4B01224A
:100EDC001A70084B1B681846FFF7E6FE054B1B689B
:100EEC0003F50073034A1360ECE700BF1400002005
:100EFC002602002028020020000000205917B7D13C
:100F0C00300600203206002080B400AF384BAA22F5
:100F1C001A80384B1B78012B30D1374B1B78012BA7
:100F2C002CD0364B1B781A46354B1988354B23F889
:100F3C001210324B1B780133DAB2304B1A702F4B34
:100F4C001B781A462A4B1B8899B22E4B23F8121089
:100F5C002A4B1B780133DAB2284B1A70284B1B88AA
:100F6C0001339AB2264B1A80244B1B78002B05D1E7
:100F7C00204B02221A70244B01221A701D4B1B7835
:100F8C00022B30D11C4B1B78022B2CD01B4B1B780B
:100F9C001A461B4B19881D4B23F81210174B1B7844
:100FAC000133DAB2154B1A70144B1B781A46104BDE
:100FBC001B8899B2154B23F81210104B1B78013378
:100FCC00DAB20E4B1A700E4B1B8801339AB20C4BD3
:100FDC001A800A4B1B78002B05D1064B01221A7084
:100FEC00094B02221A7000BFBD4680BC704700BF7F
:100FFC002C0200201A0000201B00002031060020CB
:10100C00340600203002002030060020300400207E
:10101C0080120008000000201C0000201C00002092
:10102C0038060020002103E00A4B5B584350043182
:10103C0009480A4B42189A42F6D3094A02E00023A7
:10104C0042F8043B074B9A42F9D3FFF7A5F8FFF798
:10105C001BFF704780120008000000201C000020BD
:10106C001C00002038060020FEE700000F0052E3B1
:10107C00F0402DE92900009A003081E1030013E3D0
:10108C003100001A02E0A0E110C080E2103081E2D1
:10109C00107013E50C6013E5085013E5044013E5DC
:1010AC0010E04EE20F005EE310700CE50C600CE5F6
:1010BC0008500CE504400CE5103083E210C08CE2C3
:1010CC00F2FFFF8A103042E20F30C3E30F6002E2FE
:1010DC00103083E2030056E3031081E0033080E01C
:1010EC001B00009A0140A0E106C0A0E104E043E22D
:1010FC0004C04CE2045094E403005CE30450AEE5FD
:10110C00FAFFFF8A04C046E203C0CCE304C08CE2C1
:10111C000C3083E00C1081E0032002E2000000EAB6
:10112C000030A0E1000052E30500000A013043E268
:10113C00022081E001C0D1E4020051E101C0E3E5ED
:10114C00FBFFFF1AF040BDE81EFF2FE10030A0E1CD
:10115C00F5FFFFEA0620A0E1F1FFFFEA030010E330
:10116C0010402DE93700000A000052E3012042E252
:10117C003200000AFFC001E20030A0E1020000EAE8
:10118C00000052E3012042E22C00000A01C0C3E43B
:10119C00030013E3F9FFFF1A030052E32000009A47
:1011AC00FFE001E20EE48EE10F0052E30EE88EE167
:1011BC001000009A0240A0E110C083E2104044E20B
:1011CC000F0054E310E00CE50CE00CE508E00CE536
:1011DC0004E00CE510C08CE2F7FFFF8A10C042E27D
:1011EC000FC0CCE30F2002E210C08CE2030052E3EC
:1011FC000C3083E00A00009A0340A0E102C0A0E199
:10120C0004C04CE203005CE304E084E4FBFFFF8ACF
:10121C0004C042E203C0CCE304C08CE20C3083E097
:10122C00032002E2000052E3FF100112022083109F
:10123C000200000A0110C3E4020053E1FCFFFF1A94
:10124C001040BDE81EFF2FE10030A0E1D1FFFFEA06
:10125C0000766F6C746C6F6767657200010100003B
:10126C00566F6C746C6F676765723030303000305D
:04127C00003000003E
:1012800000A24A0400000000000000000102030464
:0C129000060708090A000000FFFF010229
:0400000508001031AE
:00000001FF
